:100000009428B800841780048413A201201CA20045
:10001000102003198F28102003198F2810208F28F3
:100020003808A2060130A000A10100083805220608
:10003000031D0800A00A0319A10F15280800A60037
:100040003A0884000930A70003102B20A60CA70B48
:10005000252803142B288413B71D3A2800083804D8
:10006000371D38068000841700083804031C380642
:100070008000452800083804031C38063719380664
:1000800080008417380980054528370D0639A000FF
:100090004E20A100A00A4E200000682800308A00EF
:1000A00020088207013475340334153400343C349D
:1000B0000C34D934A301A200FF30A207031CA3070C
:1000C000031C8F280330A100DF3068205C28A101C9
:1000D000E83EA000A109FC30031C7128A00703180A
:1000E0006E28A0076400A10F6E2820187728A01C96
:1000F0007B2800007B280800A20003307F28A8008E
:1001000023082102031D8628220820020430031838
:100110000130031902302805031DFF308F28831397
:1001200003138312640008000730990083169F01AF
:1001300010308500831285018316851583120130E6
:10014000A300F4305B200230D8006400851DAA288B
:100150000230D80064008519AE28D801A00105300E
:100160008400023001202008BC002108BD003C08AA
:10017000A0003D08A100A301C8307C20031DC128B8
:10018000AE280130D90064000D3059020318DC2874
:10019000A00105308400023001202008B2002108AF
:1001A000B3000310590D3C3E840032088000840ADD
:1001B00033088000D90FC3283E08A0003F08A100E3
:1001C000A30164307C20031DE7285610E82856144C
:1001D0004008A0004108A100A30164307C20031D59
:1001E000F328D610F428D6144208A0004308A10032
:1001F000A30164307C20031DFF28561100295615E9
:100200004408A0004508A100A30164307C20031D20
:100210000B29D6110C29D6154608A0004708A100C5
:10022000A30164307C20031D172956121829561685
:100230004808A0004908A100A30164307C20031DE8
:100240002329D6122429D6164A08A0004B08A1005B
:10025000A30164307C20031D2F2956133029561723
:10026000D613D60A640056080A3C031D3829D60165
:100270004C08A0004D08A100A30164307C20031DA0
:1002800043295710442957144E08A0004F08A100D5
:10029000A30164307C20031D4F29D7105029D714A7
:1002A0005008A0005108A100A30164307C20031D68
:1002B0005B2957115C2957155208A0005308A1006B
:1002C000A30164307C20031D6729D7116829D71545
:1002D0000530BA000130B8005808B70057081F2091
:0A02E00056081F2064305A20AE2893
:02400E00C43FAD
:00000001FF
